:100000000C94DE020C94FB020C94FB020C94C81DB1
:100010000C94FB020C94FB020C94FB020C94FB026C
:100020000C94FB020C94FB020C94E4250C94B62671
:100030000C9411200C94FB020C94FB020C94FB0218
:100040000C94FB020C94FB020C94FB020C94FB023C
:100050000C94FB020C94B5200C94FB020C94FB0254
:100060000C94FB020C94FB020C94FB020C94FB021C
:100070000C94FB020C94FB020C94FB020C94FB020C
:100080000C94FB020C94FB020C94FB020C94FB02FC
:100090000C94FB020C94FB020C94FB020C94FB02EC
:1000A0000C94FB020C94FB020C94FB023C063C06F5
:1000B00068066806D006EE0606080608F9069207E6
:1000C000A307A30723274A2742284A27422896271F
:1000D000B927422810281F282200210020001F00D5
:1000E0001E00290000000000000017001500080095
:1000F0001A0014002B000000000000000A00090094
:10010000070016000400E0000000000000000500E9
:10011000190006001B001D00E100000000000000A7
:100120002C00E300E200E0000000000000000000FE
:100130000000230024002500260027002A002D00AF
:100140002E0035001C0018000C00120013004C009B
:100150002F00300031000B000D000E000F003300A7
:10016000340000005200000011001000360037007B
:100170003800E500500051004F00280002510151A5
:10018000000000000000000000000000010001006D
:10019000010001000100005C0000000000000100FF
:1001A000010001000100010001000000000000004A
:1001B0000100010001000100010001000000000039
:1001C0000000010001000100010001000100000029
:1001D000000000000100010001000100000000001B
:1001E000000000000000010001000100010001000A
:1001F0000100A800AA00A9000100010001000100FF
:1002000001000100010001000100010001000100E6
:1002100001000100010000000100000001000100D8
:1002200001000100010001000100010001000100C6
:1002300001000100010000000000000000000000BB
:1002400001000100010001000100010000000000A8
:100250000000010001000100010001000100000098
:100260000000000001000100010001000100010088
:100270000000000000000100010001000100010079
:100280000100000000000000010001000100010069
:1002900000000000000000000000010067005400A2
:1002A00055005600010001000100010001005F003F
:1002B0006000610057000100010001000100010021
:1002C0005C005D005E000100010000000100000014
:1002D000010059005A005B0001000100010001000B
:1002E0000100010001006200630000000000000046
:1002F0000000000044454255473A2064697361623A
:100300006C65642E0A0044454255473A20656E618B
:10031000626C65642E0A000A0025303258006C6554
:10032000645F7461736B3A20004F6E6573686F741D
:100330003A206163746976653A2025640A000A00F0
:100340002530313662003A200025303258000A72DA
:100350002F63203031323334353637383941424318
:100360004445460A0054617267657420636F6E6E7F
:1003700065637465640D0A00546172676574206476
:100380006973636F6E6E65637465642C2074687244
:100390006F74746C696E6720636F6E6E65637469E9
:1003A0006F6E20617474656D7074730D0A00466120
:1003B000696C656420746F20657865637574652069
:1003C00025730A00290A002575002F002575005D98
:1003D00028002564002000256400200025640020FA
:1003E000002564007C0025303258006D6F75736500
:1003F0006B6579205B62746E7C782079207620684A
:100400005D287265702F61636C293A205B000A00D9
:100410002530325820006B6579626F6172645F72BB
:1004200065706F72743A20005B735D005B575D000E
:100430005B535D005B525D005B445D005B435D00B0
:100440000E0342007200650065007A00650000003E
:100450001C03410066007400650072006E006F00AE
:100460006F006E004C006100620073000000040326
:10047000090409025B00030100A0FA09040000015D
:10048000030101000921110100012240000705813B
:100490000308000109040100010300000009211103
:1004A000010001227B0007058203200001090402EC
:1004B00000020300000009211101000122220007AF
:1004C000058303200001070503032000011201003A
:1004D00002000000086C6101000100010200010639
:1004E00031FF0974A1010975150026FF00952075DB
:1004F0000881020976150026FF00952075089102F3
:10050000C005010902A10185020901A1000509191F
:1005100001290815002501950875018102050109C9
:100520003009311581257F95027508810609381536
:1005300081257F950175088106050C0A3802158111
:10054000257F950175088106C0C005010980A101BC
:10055000850319012AB700150126B700950175100A
:100560008100C0050C0901A101850419012AA0021E
:10057000150126A002950175108100C0050109062C
:10058000A101050719E029E7150025019508750166
:1005900081029501750881010507190029FF1500E1
:1005A00026FF0095067508810005081901290595A3
:1005B0000575019102950175039101C011241FBEBB
:1005C000CFEFDAE0DEBFCDBF11E0A0E0B1E0E6E3BF
:1005D000F2E502C005900D92AC3CB107D9F723E0DB
:1005E000ACECB1E001C01D92A531B207E1F70E9469
:1005F000B7170C9419290C940000FF93EF93E09126
:10060000CC01F091CD01309709F00995EF91FF9160
:100610000895FC018591803011F0EFDFFBCF089544
:10062000FF27E0E230E247FF0CC0419597FF09C089
:10063000EDE26095709580959095611D711D811D0D
:10064000911D27FF02C0219530E350E2AA27660FD3
:10065000771F881F991FAA1FA41710F0A41B63956A
:100660005A95A9F7AA3008F0A95FA05DAF93F3955A
:10067000611571058105910541F7ED3211F4EF9394
:10068000F395F21718F43F93F395FBCF8F91B5DFF5
:10069000FA95E1F70895E991F9918591803021F07B
:1006A000853219F0AADFF9CF089520E0E89455913A
:1006B0005532C1F3503311F4689455915A3348F4CC
:1006C000505390F3220F022E220F220F200D250FE0
:1006D000F4CF0EF4219589919991533619F353373C
:1006E00029F1533559F1BC0188279927E8945C36E4
:1006F00021F48991999168945591543639F446EFD3
:100700007EF077FF0DC08FEF9FEF0AC055374AE0AC
:1007100039F0583540E121F0523642E009F00895B1
:10072000FF93EF937DDFEF91FF91B7CFFF93EF93AF
:10073000FC0181918030B9F360DFFBCFFF93EF9331
:1007400068DFF1CFDF93CF93CDB7DEB72596A3DF78
:10075000CF91DF91089581E0089581E008950C9490
:10076000AD0308950C94B1031F93CF93DF9300D092
:1007700000D01F92CDB7DEB749835A836B83309187
:10078000CF0189819A81311114C0662359F0222347
:1007900049F00E94430A182F682F89819A810E948C
:1007A000EC0903C00E94170A182F69817A81812FF2
:1007B00004C00E94430A69817A810F900F900F90C4
:1007C0000F900F90DF91CF911F910C949511FC0128
:1007D000262F408151816281738184810C94B403FE
:1007E00081E00895CF93DF93EC0160E00E94E7037E
:1007F000BE01DF91CF910C94B2030C9473130C944F
:100800006F1308950E9496080E9401042FEF84E35D
:100810009CE0215080409040E1F700C000000C9423
:10082000DB200F931F93CF93DF938C0161E00E9435
:10083000E703EC01B8010E94AF03882309F45BC011
:10084000B801CE010E94D31C882309F454C0B8011A
:10085000CE010E94E71A882309F44DC0B801CE01E9
:100860000E942F1C882309F446C0F8018281882346
:10087000D9F1CF3D8CE5D80779F140F4C115FCE5FD
:10088000DF0791F0C130DC4591F02EC0CC35EDE5AD
:10089000DE0741F1CD35FDE5DF0709F1CB35DD455B
:1008A00019F50E94DA0E20C00E94020424C0809133
:1008B0007C02C82FC095C170C0FB80F980937C0278
:1008C000CC2329F086E093E00E94090314C084EF52
:1008D00092E00E94090310C00E948E0F0CC00E947B
:1008E000D10E02C00E94DD0EC801DF91CF911F9191
:1008F0000F910C94AB03C0E08C2FDF91CF911F912F
:100900000F9108950E94F31F0C94C0040E94C30429
:100910000C94F91F8295982F937344E0949F900153
:1009200011248C7C86958695282B822F8575880FBF
:100930002A7A2695822B0895CF93DF93D92F0E9490
:100940008A04C82F8D2F0E948A042C2F30E0322F6A
:100950002227A901482BCA01DF91CF91089508955C
:100960000C94AF0481E008950C94B2040895CF93E1
:10097000C82F0E94B0048C2F0E94B404CF91089518
:1009800080E00C94B7040E94F31E0C94B704CF933C
:100990000E94F31EC82F8091CE01C81741F1C09369
:1009A000CE0180917C0282FF1EC080FF04C08EE1D8
:1009B00093E00E94090380917C0280FF0CC01F928B
:1009C000CF9389E193E09F938F930E94A2030F90AE
:1009D0000F900F900F9080917C0280FF04C087E100
:1009E00093E00E9409038C2FCF910C94B704CF9110
:1009F0000895CF93DF93CDB7DEB72B970FB6F8945A
:100A0000DEBF0FBECDBF4F83588769877A878B873C
:100A100061110E94090E9E012F5F3F4F86E0F90190
:100A200011928A95E9F785E0FE013796D901019088
:100A30000D928A95E1F789819A814C815D81452BE0
:100A400031F09F3F31F491E08F3F19F403C091E002
:100A500001C090E090FF09C049815A816B817C817F
:100A60008D819E810E942A0D05C0C9010E94F0035C
:100A70008111F2CF2B960FB6F894DEBF0FBECDBF1B
:100A8000DF91CF910895FC01808191810E94850AB8
:100A90000895CF93882309F450C0C82F8CEF8C0F92
:100AA000813AD0F46C2F80910201909103010E9451
:100AB000951F882349F06C2F8091020190910301CA
:100AC0000E94CD1F0E942B0E6C2F809102019091ED
:100AD00003010E94CB1F0CC080E28C0F883058F4B9
:100AE000C77081E001C0880FCA95EAF70E94EC0D3B
:100AF000CF910C942B0EEBE5EC0FE33040F4F0E0DB
:100B0000E05AFE4F808190E0CF910C945D1FE8E5A4
:100B1000EC0FE73150F4F0E0EE0FFF1FEE5CFE4FFC
:100B200080819181CF910C94731FCD3E30F08C2F3A
:100B30000E943C18CF910C940E19CF9108958823F0
:100B400089F19CEF980F913A40F4682F809102014F
:100B5000909103010E94CD1F0DC090E2980F983034
:100B600058F4877091E001C0990F8A95EAF7892FB0
:100B70000E94F20D0C942B0E9BE5980F933020F4FD
:100B800080E090E00C945D1F98E5980F973120F479
:100B900080E090E00C94731F8D3E20F00E94971827
:100BA0000C940E1908951F93CF93DF93182FEB0128
:100BB0000E944905209741F08FE99FE00197F1F7E6
:100BC00000C000002197F6CF812FDF91CF911F91B8
:100BD0000C949F05893319F060E070E002C060E575
:100BE00070E00C94D305882321F00E94EC0D0C9446
:100BF0002B0E0895882321F00E94F20D0C942B0EE9
:100C00000895CF92DF92EF92FF920F931F93CF93AD
:100C1000DF937C01D62FC72FFC011281058102953D
:100C20000F700E94E20D8823B9F01123A9F08C2FD8
:100C3000807F803421F080E28D0F883068F08091D1
:100C4000D90282FD09C082E00E948B0E0E94E20D53
:100C500091E0D82ED92601C0D12CCC2EC2948FE0A1
:100C6000C8228C2D90E08C30910508F0CFC1FC019A
:100C7000EA5AFF4F0C94A7288C2F807FCF708823CF
:100C800011F0C295C07F112399F0CC2309F4AAC1B9
:100C900080E28D0F883010F0D11104C08C2F0E949B
:100CA000EC0D03C08C2F0E94FC0D0E942B0E9AC1EC
:100CB0008D2F0E949F05CC2309F4A8C180E28D0FDF
:100CC000883038F1DD2329F18C2F0E94020E24C0D8
:100CD0008C2F807FCF70803211F0C295C07FDD23D2
:100CE00019F0D130A1F13DC08091D90282FF17C027
:100CF000112349F0CC2329F08C2F0E94EC0D0E9487
:100D00002B0E80E070C180E00E949F05CC2309F487
:100D10007DC18C2F0E94F20D0E942B0E77C11123F2
:100D200071F0002341F0013031F40E940C0E8C2B45
:100D30000E94140E6BC10E940C0E8C2B1DC0002350
:100D400019F0013009F462C10E94210E25C011235F
:100D500021F0063008F05AC10EC0053008F056C127
:100D60001BC0112361F0002331F0F701858180FF62
:100D700039C18F7085838C2F0E94F30547C10023F2
:100D800059F0D93309F03FC1FFEF07EE13E0F150FE
:100D900000401040E1F735C18C2F0E94FA0536C1A2
:100DA0008C2F86958695837019F0813061F02EC165
:100DB000112321F08D2F9C2F937002C080E090E0D2
:100DC0000E945D1F2BC1112321F08D2F9C2F93704A
:100DD00002C080E090E00E94731F20C18D2F11237C
:100DE00019F00E943C1802C00E9497180E940E1928
:100DF00015C18C2F837009F047C011110BC12D2F25
:100E0000229526952770220F220F6D2F6F70862F47
:100E100090E0A0E0B0E0022E04C0880F991FAA1F46
:100E2000BB1F0A94D2F7D4FF10C04FE050E060E03F
:100E300070E004C0440F551F661F771F2A95D2F734
:100E4000409550956095709503C040E050E0BA0120
:100E5000C695C695C3708A019B01082B192B2A2BB6
:100E60003B2BC901B801C23049F058F4C13019F028
:100E70000E940209CFC00E94F008CCC00E94140951
:100E8000C9C00E94EE08C6C0112319F08C2F8170D2
:100E900001C08695882309F4BDC02D2F2295269583
:100EA0002770220F220F6D2F6F70862F90E0A0E029
:100EB000B0E0022E04C0880F991FAA1FBB1F0A941E
:100EC000D2F7D4FF10C04FE050E060E070E004C003
:100ED000440F551F661F771F2A95D2F740955095EE
:100EE0006095709503C040E050E0BA01C695C69584
:100EF000C3708A019B01082B192B2A2B3B2BC9019C
:100F0000B801C23049F058F4C13019F00E94C70945
:100F100081C00E94B5097EC00E94D9097BC00E9491
:100F2000280978C0CF70112339F08C2F0E944E0908
:100F30008D2F0E94F3056EC08D2F0E94FA058C2F15
:100F40000E946F0967C0D23F21F128F4D03F41F0E1
:100F5000D13FC1F043C0D33F19F1D43F79F03EC037
:100F6000112341F0053008F051C08C2F8F710E9481
:100F700094094CC0063008F049C0F7CF8091D902DF
:100F800082FF18C0112339F08C2F8F710E944E09F7
:100F90003DC01123C9F38C2F8F710E946F0936C099
:100FA000112329F08C2F8F710E9439092FC00E94C4
:100FB00034092CC0112349F0CF718C2F0E944E09A7
:100FC00063E08C2F0E94700E21C081E00E948B0E86
:100FD0000230E0F082E00E948B0E18C0112331F045
:100FE000002391F28D2F0E94490510C0002399F231
:100FF000D93349F41FEF27EE33E011502040304041
:10100000E1F700C000008D2F0E949F0588EF8C0D36
:10101000843020F40E94F31E0E94B704DD20C9F042
:101020000E94DE0D80FD15C0F70112820E94D80DCE
:101030000E944E09C7010E944A080E94D80DDF9104
:10104000CF911F910F91FF90EF90DF90CF900C9474
:101050006F09DF91CF911F910F91FF90EF90DF907B
:10106000CF9008950F931F93CF93DF93EC01688186
:1010700079818A810E94900A8C010E94EB090E946A
:10108000DC08B801CE010E940106DF91CF911F91CB
:101090000F910895CF93DF93EC01988189812B8183
:1010A0003C81232B31F08F3F31F481E09F3F19F4D5
:1010B00003C081E001C080E080FD1DC0CE010E9420
:1010C0001104811110C00E94E20D8823A1F08A81D1
:1010D000882389F08091D90282FD0DC082E0DF91E2
:1010E000CF910C948B0ECE010E943208CE01DF917D
:1010F000CF910C94F203DF91CF91089580E090E0BE
:101100000E945D1F80E090E00E94731F0E94090E04
:101110000E942B0E0E94C11A0C940E19809102019C
:10112000909103010E94CF1F0C947E080E94F90D3C
:101130000C948E0892959F70963079F010F492502E
:1011400001C09A50923068F4803F69F018F4883EEC
:1011500040F409C0843F29F406C0883E20F0813F56
:1011600011F080E0089581E00895FC018081918173
:101170000E94850A0E949A080895CF93DF9300D0B9
:1011800000D01F92CDB7DEB70F900F900F900F9049
:101190000F90DF91CF910895CF93DF9300D000D0CF
:1011A00000D0CDB7DEB726960FB6F894DEBF0FBEDF
:1011B000CDBFDF91CF910895089508950C94DD0877
:1011C0000C94DE080E94E0086093100270931102F4
:1011D00080931202909313020C947E080C94E20800
:1011E0000F931F930091100210911102209112028F
:1011F00030911302602B712B822B932B1F910F9137
:101200000C94E2080F931F930091100210911102A9
:1012100020911202309113026023712382239323C1
:101220001F910F910C94E2080F931F9300911002ED
:101230001091110220911202309113026027712740
:10124000822793271F910F910C94E2080C94DD08DC
:101250000E94260960930C0270930D0280930E0287
:1012600090930F020C947E0860E070E0CB010C9428
:1012700028090F931F9341E050E060E070E08A017D
:101280009B0104C0000F111F221F331F8A95D2F744
:10129000C901B8011F910F910C9428090F931F9356
:1012A00041E050E060E070E004C0440F551F661F4D
:1012B000771F8A95D2F780910C0290910D02A09130
:1012C0000E02B0910F028A019B01082B192B2A2BC9
:1012D0003B2BC901B8011F910F910C9428090F9362
:1012E0001F9341E050E060E070E004C0440F551FE0
:1012F000661F771F8A95D2F7409550956095709537
:1013000080910C0290910D02A0910E02B0910F02FB
:101310008A019B01082319232A233B23C901B80111
:101320001F910F910C9428090F931F9341E050E0F7
:1013300060E070E004C0440F551F661F771F8A9558
:10134000D2F780910C0290910D02A0910E02B09103
:101350000F028A019B01082719272A273B27C90169
:10136000B8011F910F910C9428090F931F930091BE
:101370000C0210910D0220910E0230910F02602B91
:10138000712B822B932B1F910F910C9428090F9393
:101390001F9300910C0210910D0220910E023091CA
:1013A0000F0260237123822393231F910F910C94CA
:1013B00028090F931F9300910C0210910D022091A8
:1013C0000E0230910F0260277127822793271F9109
:1013D0000F910C942809089529E0929F800D112403
:1013E000E82FE695E695E695877051E001C0550F28
:1013F0008A95EAF785E0E89FF0011124E053FE4F5B
:1014000020E030E070E04081CB01022E02C09695D2
:1014100087950A94E2F78170819584278523842734
:1014200081932F5F3F4F2530310569F7089529E0FB
:10143000929F800D1124682F669566956695982F6A
:10144000977085E0689FB001112440E050E080E093
:10145000FB01E40FF51FE053FE4F208130E0092E21
:1014600002C0369527950A94E2F721703327042E9F
:1014700001C0220F0A94EAF7822B4F5F5F4F45307D
:10148000510531F70895BF92CF92DF92EF92FF920C
:101490000F931F93CF93DF938C01C0900C02D090D9
:1014A0000D02E0900E02F0900F02809110029091D8
:1014B0001102A0911202B0911302C82AD92AEA2A75
:1014C000FB2ACFE1D0E0D701C6010C2E04C0B695AF
:1014D000A795979587950A94D2F780FD04C0219728
:1014E00090F7B12C07C0BC2EB8018C2F0E94A81118
:1014F0000197A9F38B2DDF91CF911F910F91FF9051
:10150000EF90DF90CF90BF900895CF93DF93EC01E1
:101510000E94430ABE010E94A811DF91CF91089555
:101520001F93CF93DF93EB019091CF01992321F08B
:10153000CB010E94850A13C0882349F0CB010E9489
:10154000430A182F682FCE010E94EC0904C0CB017A
:101550000E94170A182FBE01812F0E94A811DF9147
:10156000CF911F9108951F93CF93DF93C0911402E1
:1015700016E080911502C81799F0D0E01C9FF00189
:101580001D9FF00D1124EA5EFD4F40815181628163
:101590007381848195810E94CC082196C770E9CF20
:1015A000DF91CF911F9108954091460250914702DB
:1015B000609148027091490280914A0290914B02D9
:1015C0000C94CC08EF92FF920F931F93CF93DF936D
:1015D00080914B0282958F7009F065C0809148021E
:1015E000882309F460C080911402F09015021091D4
:1015F0004602009147026091490270914A0291E0CF
:101600001F3F09F090E0C0910001D0910101292F06
:1016100096E0E92E8F1509F446C06115710521F099
:101620000F3F21F030E003C031E001C0322F90E0E5
:1016300030FD36C0E89EF001E99EF00D1124DF0177
:10164000AA5EBD4F11963C911197301329C03C9171
:10165000311326C012963C911297311121C0139676
:101660004D915C911497461B570B4C175D07C0F4C6
:1016700080914B028F70806180934B02E55EFD4F3D
:1016800080818F708061808386E492E00E944A08A6
:10169000DF91CF911F910F91FF90EF900C94B30ABF
:1016A00001968770B7CFDF91CF911F910F91FF9077
:1016B000EF9008959F92AF92BF92CF92DF92EF92F8
:1016C000FF920F931F93CF93DF93CDB7DEB7619750
:1016D0000FB6F894DEBF0FBECDBF8C0185E0F801D8
:1016E000DE011D9601900D928A95E1F7D8011296C0
:1016F000EC9090914602E09147022091490230918E
:101700004A022115310531F0EF3F31F481E09F3F6E
:1017100019F403C081E001C080E0B82FB1709B2EA6
:1017200080FD47C1D8014C9111965C911197139699
:10173000AD90BC90149786E4C82E82E0D82EF0902D
:101740004802B501621B730B209100013091010129
:10175000FF2009F4D9C080914B026217730708F08B
:1017600095C0282F207F09F052C05E1313C0491383
:1017700011C0FE2CE1100EC08F70806180934B026F
:101780000E94D40AC6010E944A0880914B02F801C7
:1017900085834DC1AB2831F05F3F31F481E04F3F8D
:1017A00019F403C081E001C080E080FD03C081E046
:1017B0008E2502C080E090E0F82FF170FF2E80FFB0
:1017C0001CC0809114022091150236E0821709F4A2
:1017D0000BC190E0389FF001399FF00D1124EA5EB3
:1017E000FD4F6181561306C06081461303C06281BC
:1017F000E61203C001968770E9CFFE2CEE2009F4B3
:1018000016C180914B02816080934B0254C05E13DD
:1018100006C0491304C0E11002C0F80199C0C80114
:101820000E94B508882361F1EE2051F120914B020E
:10183000822F82958F7090E0029774F0809146021B
:101840009091470298878F831986BB86AA862C873A
:10185000CE0107960E944A0886E0F801A6E4B2E0AD
:1018600001900D928A95E1F70E94E20A0E94D40A43
:101870000AC05E1711F1C8010E94B50881112CC081
:10188000C8010E944A08FF24F394D1C0282F207F6A
:1018900081F77A2DB98AA88A6E2D89890E94BD08A0
:1018A00086E492E00E944A0886E0D6011D928A955D
:1018B000E9F70E94D40AF12CBAC04913DCCFE11039
:1018C000DACFF8018583C8010E944A0886E0D60174
:1018D0001D928A95E9F7ABC0EE2091F220914B0260
:1018E000822F82958F7090E002970CF4B5CF809193
:1018F0004602909147029A8389831B82BD82AC8203
:101900002E83CE010196A6CF6217730708F044C05C
:10191000FE2CEE2009F4B4CF5E1330C049132EC064
:1019200020914B0220FD21C0822F82958F70482F7D
:1019300050E041155105C9F0F80125834F3051059C
:1019400041F08F5F982F9295907F822F8F70892B17
:101950008583C8010E944A0886E0F801A6E4B2E047
:1019600001900D928A95E1F73CC086E0F801A6E46B
:10197000B2E001900D928A95E1F759C0C8010E942A
:10198000B508811169CF80914B02816080934B0231
:10199000C8010E944A084BC07A2DB98AA88A6E2DC8
:1019A00089890E94BD0886E0D6011D928A95E9F7D3
:1019B00018C0EE2009F464CFC8010E94B508F82EC3
:1019C000882309F45DCF86E0F801A6E4B2E0019037
:1019D0000D928A95E1F786E492E00E9443050E9409
:1019E000E20A0E94D40A23C04D875E878D859E85BA
:1019F0000E94850A292F22952F70223028F49F708B
:101A000039F0811105C00BC0243028F49F7049F4CF
:101A1000805E883020F0C8010E944A089F2CF92C73
:101A200006C0D80115969C91907F91F7F8CF8F2D25
:101A300061960FB6F894DEBF0FBECDBFDF91CF9198
:101A40001F910F91FF90EF90DF90CF90BF90AF90DC
:101A50009F9008951F93CF93DF93CDB7DEB72C9758
:101A60000FB6F894DEBF0FBECDBF4F83588769878E
:101A70007A878B879C87CE0107960E945A0B882312
:101A8000D1F09F8188852A853B85232B31F08F3FBC
:101A900031F481E09F3F19F403C081E001C080E090
:101AA00080FD47C04F81588569857A858B859C85E7
:101AB0000E94CC083EC086E0FE013796DE011196FA
:101AC00001900D928A95E1F7FF81E8856A857B8513
:101AD0006115710531F0EF3F31F481E0FF3F19F4FA
:101AE00003C081E001C080E080FD23C02091150289
:101AF00030E0C9010196877099274091140250E0A7
:101B000084179507F1F1F983EA837D836C8396E06E
:101B1000929FD001939FB00D1124AA5EBD4FFE018C
:101B2000319601900D929A95E1F7809315020E94EB
:101B3000B30A16E08091140290911502891771F191
:101B4000189FC00111248A5E9D4F0E945A0B882362
:101B500029F1E09114021E9FF0011124EA5EFD4F6D
:101B60004081518162817381848195810E94CC087A
:101B70008091140290E00196877099278093140257
:101B8000D9CF0E9496081092150210921402E6E432
:101B9000F2E086E0DF011D928A95E9F72C960FB6F8
:101BA000F894DEBF0FBECDBFDF91CF911F91089596
:101BB000809154028595859585950895809154026C
:101BC0008770089590915402977081E009F480E045
:101BD000089580915F02089590915F02892B809310
:101BE0005F020895809590915F02892380935F0240
:101BF000089510925F02089590915E02892B809360
:101C00005E020895809590915E02892380935E0222
:101C1000089510925E0208958091550208950895E6
:101C20000C940F0E0C94100E9091D90292FD08C0E6
:101C300090915502981721F0809355020C94120E42
:101C4000089580915502882329F01092550280E072
:101C50000C94120E0895CF93DF93E0910201F0915E
:101C6000030180915F028083E0910201F091030102
:101C7000908180915E02892B808380915502882318
:101C800081F0E0910201F09103019081892B808322
:101C900080910201909103010E94891F81110E948D
:101CA000210EC0910201D091030148E050E06CE4A4
:101CB00072E0CE010E94C128892B69F088E0FE0104
:101CC000ACE4B2E001900D928A95E1F7CE01DF918C
:101CD000CF910C94061FDF91CF9108950C940F0EB5
:101CE0009091D90292FD10C098E0899F9001112433
:101CF000262B209354020E944E0980915402859510
:101D0000859585950C946E0E0C944E091092540294
:101D100080E00C946E0E2091540280958223809373
:101D20005402982F977099F430E0482F082E000C39
:101D3000550B2417350759F09091D90292FD07C031
:101D40008595859585950E946F090C94860E08955A
:101D5000CF939091D90292FB222720F92817F9F00E
:101D6000C82F892FC0FB82F98093D9028091D802B5
:101D70009091D9020E940A0F82E00E948B0E8091FE
:101D80007C0280FF0CC01F92CF9389E293E09F9367
:101D90008F930E94A2030F900F900F900F90CF91FE
:101DA00008958091D90282FB882780F991E08927E4
:101DB0000C94A80E81E00C94A80E80E00C94A80E60
:101DC0006FEF7FEF80E090E00C94032980E090E0DB
:101DD0000E94DF2821E0893E9E4F09F020E0822FFB
:101DE000089582E090E00C94D72883E090E00C9472
:101DF000D728CF9384E090E00E94D728C82F82E2B2
:101E000090E00E94D7282C2F30E0A901582BCA015E
:101E1000CF910895CF93C92F682F84E090E00E945E
:101E2000E5286C2F82E290E0CF910C94E528AB017D
:101E3000BC018FE090E00C94F728AB01BC0183E17A
:101E400090E00C94F72860E070E0CB010C941D0F3B
:101E500060E070E0CB010E94170F0C94230F69EE35
:101E60007EEF80E090E00E94032960E082E090E055
:101E70000E94E52860E083E090E00E94E52810924F
:101E8000100210921102109212021092130260E0DE
:101E900084E090E00E94E52860E082E290E00E9409
:101EA000E52860E085E090E00E94E52860E086E0BB
:101EB00090E00E94E5286FEF87E090E00E94E5281F
:101EC00040E050E0BA0188E090E00E94F72860E02E
:101ED0008DE090E00E94E52840E050E0BA0188E102
:101EE00090E00E94F72860E087E190E00E94E528FA
:101EF00040E050E0BA018CE190E00E94F72860E0F9
:101F000070E080E290E00E94032940E050E0BA01D6
:101F100088E190E00E94F7280C94280F0C942F0F72
:101F2000682F8EE090E00C94E5280E947E2060935C
:101F300078027093790280937A0290937B02609387
:101F400074027093750280937602909377020895DD
:101F500085B7806885BF85B7806885BF08950C9474
:101F60004E1508950C94B10F0C94B10F0C94B40F4E
:101F70000C94B10F0C94B80F0C94B10F0E94A80FE1
:101F80008FEB92E20E94E91E0E94BC0F0C94BA0FE4
:101F90000E94B20F0C94B10F0E94F0120C94B60480
:101FA0000E9469200E9484120E9466150E94921469
:101FB0000E94CC0F0E94CF1A0E9470150C94B60F8D
:101FC0005F926F927F928F929F92AF92BF92CF92C9
:101FD000DF92EF92FF920F931F93CF93DF93CDB7D2
:101FE000DEB72A970FB6F894DEBF0FBECDBF0E94B2
:101FF000B614C82E81110E94950F30E6832E32E070
:10200000932E00E010E0502E802F0E9414135C01EC
:10201000F401619071904F01682679266114710472
:10202000B1F40F5F1F4F0A30110569F78FEF8983F5
:102030008A831B820E9472208160782F9D838C830B
:1020400049815A816B818D810E94F9043AC0809147
:102050007C0281FD0E941D13D12CEE24E394F12C0F
:10206000C3018E219F21892B29F10E94AF0F882364
:10207000A9F0DE825F82AE20BF2081E0AB2809F4A8
:1020800080E088870E9472208160782F9A878987F4
:102090004E815F8168858A850E94F904000F111FB7
:1020A000F801E05AFD4F80819181E826F926F182FE
:1020B000E08207C0D394EE0CFF1CF9E0DF12D0CF12
:1020C000B0CF81E0C11001C080E02A960FB6F8942D
:1020D000DEBF0FBECDBFDF91CF911F910F91FF905B
:1020E000EF90DF90CF90BF90AF909F908F907F90B8
:1020F0006F905F9008950E94E00F0E944E150E941D
:10210000AE190C94C704CF93DF930E94AD11EC017C
:10211000811521E5920708F045C0811530E5930748
:1021200008F094C0883E910528F5803E910508F09E
:10213000F8C0883A910570F4853A910508F07CC0A2
:102140008130910509F475C008F4E8C0049708F0DF
:10215000E8C0E4C08F3B910508F0E0C0C85AD0E069
:10216000CC0FDD1FCD59DE4F0990D881C02DCE0197
:102170009464D8C0811540E2940758F4811551E069
:10218000950708F0CEC08D3E910508F4C7C0906554
:10219000C9C0C11580E4D80708F4C0C0DF70CE0103
:1021A000906AC0C0811525E59207A8F4811534E531
:1021B000930708F095C0811543E5940708F07BC0AC
:1021C000811552E5950708F061C0D82FCC27CE01C4
:1021D000816F906AA7C0C11589E5D807A0F4C11521
:1021E00028E5D20708F082C0C11536E5D30708F00C
:1021F00095C08C2F0E9441128F7190E0D82FCC2770
:10220000CE0190628FC0C1154AE5D40708F474C0AE
:10221000CE0190568115904208F080C08D2F8F71AD
:102220000E944112DD27D0628F71AE01582BCA0186
:1022300079C081E090E076C0C55AD0E0CF56DE4F3D
:102240008881C82FD0E0CE0190646CC074E0969570
:1022500087957A95E1F7282F23703C2F337081E022
:1022600090E002C0880F991F3A95E2F79C68AC0194
:10227000522B9A019C2F9F709695969550E2959FB0
:10228000E0011124C9018C2B9D2B4CC08370992730
:1022900021E030E002C0220F331F8A95E2F79C2F25
:1022A0009695969580E2989FE0011124C22BD32B3E
:1022B000CE019C6837C08370992721E030E002C0CE
:1022C000220F331F8A95E2F79C2F9695969540E250
:1022D000949FE0011124C22BD32BCE019A6822C017
:1022E000D82FCC27CE01846F906A1CC0DC2FCC275E
:1022F000CE01806F906A16C08C2F8F700E944112A1
:1023000094E0D695C7959A95E1F7CF70D0E0DC2F91
:10231000CC27D0699E01282BC90104C080E090E041
:1023200001C0CE01DF91CF9108952AE5829FC001BF
:102330001124FC0129E0729FE00DF11D1124E60F2C
:10234000F11DEE0FFF1FE852FF4F85919491089504
:102350000E9495110E94831008958238910569F1B9
:10236000B0F48133910509F46DC048F489329105C8
:1023700009F463C08A32910509F469C00895853370
:10238000910509F455C089339105B9F00895833E4C
:10239000910569F138F4803E9105B1F0823E9105D6
:1023A00009F10895863E9105A9F1873E9105B9F19D
:1023B000843E910509F064C023C02091D80220FD1D
:1023C0004FC021FD4DC008958091D80280FD44C0CA
:1023D0008091D90280FF44C08091D80284FD42C020
:1023E00083EE4DC08091D80282FF38C0F5CF809136
:1023F000D80282FD33C08091D90280FD31C0ECCF7C
:102400008091D90281FF32C08091D80284FD2AC018
:1024100087EE35C08091D80283FF26C0F5CF80912A
:10242000D80283FD21C08091D90281FD1FC0ECCF6D
:102430008091D80285FD1CC01DC08091D80285FD09
:1024400019C016C08091D80286FD16C017C08091B1
:10245000D80286FD13C010C089E311C082EE0FC000
:1024600080EE0DC080E00BC086EE09C084EE07C090
:1024700089E205C085E303C08AE201C081E390E000
:1024800008959091D80292FF0DC0282F287128300E
:1024900019F4877F846006C0282F2471243011F43A
:1024A0008B7F886093FF0DC0282F2871283119F485
:1024B000877E846106C0282F2471243111F48B7E1D
:1024C00088612091D90220FF0DC0382F3871383033
:1024D00019F4877F816006C0382F3171313011F4D3
:1024E0008E7F886021FF0DC0282F2871283119F4B4
:1024F000877E816106C0282F2171213111F48E7EE3
:10250000886194FD877E08951092D4021092D502BE
:102510001092D6021092D7020895CF92DF92EF92D6
:10252000FF926B017C010E944E1581110EC00E942A
:102530007E20C61AD70AE80AF90AC092D402D092BD
:10254000D502E092D602F092D702FF90EF90DF9092
:10255000CF9008950F931F930E944E15882321F06A
:102560001F910F910C947E200E947E200091D40236
:102570001091D5022091D6023091D702600F711FC1
:10258000821F931F1F910F9108950C94E00ECF931B
:102590000E94B6148FE39CE90197F1F700C0000098
:1025A0000E94B6140E944715811102C0C5E001C007
:1025B000C0E080E00E94141321E030E002C0220F4E
:1025C000331FCA95E2F782239323892B29F00E94B7
:1025D000C512CF910C94DB20CF9108950C94C712B3
:1025E0000E94E60E811102C00E948E0F0E94F10E21
:1025F00080937C020E94F90E9093D9028093D802B6
:102600000E94EE120E94F50E682F70E080E090E0CC
:102610000E94EE0860910C0270910D0280910E02F2
:1026200090910F020C942609E82FF0E0EE0FFF1FA7
:10263000E151FD4F808191810895CF92DF92EF9219
:10264000FF920F931F93CF93DF938EE493E00E944A
:1026500009038FEEE82E82E0F82EC0E0D0E099E486
:10266000C92E93E0D92E00E413E0DF93CF93DF92DD
:10267000CF920E94A20386E493E00E940903F7012F
:10268000819191917F010E949C049F938F931F934E
:102690000F930E94A2038EE393E00E940903219608
:1026A0008DB79EB708960FB6F8949EBF0FBE8DBF2C
:1026B000CA30D105D1F6DF91CF911F910F91FF90D4
:1026C000EF90DF90CF90089580EA8A95F1F7089512
:1026D00000C008950C94641308950C946C130C942A
:1026E0006D130C946C130C9471130C946C13FF9277
:1026F0000F931F93CF93DF93CDB7DEB72A970FB613
:10270000F894DEBF0FBECDBF0E944E15609103034B
:10271000882309F443C05AE0F52E8E010F5F1F4F46
:10272000F8018F2D11928A95E9F7862F90E0880F96
:10273000991FB80181519D4F0E947E15882399F001
:102740008091DA0290E0880F991F4AE050E0B801CA
:1027500081519D4F0E94C12821E020937D02892B49
:1027600061F410E018C080917D028823D1F3F80154
:102770001192FA94E9F710927D02A091DA02B0E08A
:10278000AA0FBB1FA151BD4F8AE0F80101900D9225
:102790008A95E1F711E00E94FF0311C08091DA02EF
:1027A00070E0660F771F61517D4F90E0880F991F91
:1027B00081519D4F0E941A160E94751310E0812FBF
:1027C0002A960FB6F894DEBF0FBECDBFDF91CF9132
:1027D0001F910F91FF900895F894E82FE295EF7004
:1027E000F0E031A1282F2F7081E090E001C0880F28
:1027F0002A95EAF7982F9095932391A392A1892B7C
:1028000082A3789408950F931F93CF93DF93CDE91C
:10281000D1E089918F3F11F00E94EC1381E0C23A20
:10282000D807B9F7C4E9D1E00DE911E089918F3FEC
:1028300011F00E94EC130C171D07C1F7DF91CF9127
:102840001F910F910895BF92CF92DF92EF92FF9266
:102850000F931F93CF93DF938C01C62FD0E0CE014F
:1028600083569E4F6C01FC0190819F3F09F450C03C
:10287000B62EF894E92FE295EF70F0E081A19F70F9
:1028800021E030E001C0220F9A95EAF7822B81A364
:1028900082A12095282322A378940E946813E4E95A
:1028A000F1E04DE951E021E030E0E12CF12C6191C3
:1028B0006F3F89F0A62FA295AF70B0E090968C91F3
:1028C00090E06F7002C0959587956A95E2F780FD5C
:1028D00002C0C90102C080E090E0E82AF92A220F74
:1028E000331F4E175F0719F7F60180818F3F11F0F4
:1028F0000E94EC1361E0E114F10409F460E08B2D17
:102900000E946A13CC0FDD1FC00FD11FF982E8822D
:10291000DF91CF911F910F91FF90EF90DF90CF90BB
:10292000BF9008958091040180910401811102C03B
:1029300095E001C090E09093030385E0891B8093AC
:10294000DA020E94031484E1EFEEF2E0DF01982F37
:102950001D929A95E9F7EBEDF2E0DF011D928A9561
:10296000E9F785E00E940C150C94FD03EF92FF92AD
:102970000F931F93CF93DF93CDB7DEB764970FB656
:10298000F894DEBF0FBECDBF8E010F5F1F4F84E1F5
:10299000F80111928A95E9F7F12C6F2DC8010E9478
:1029A0002314F394F5E0FF12F8CF44E150E0B801AE
:1029B0008BED92E00E94C1287C0121E0892B09F473
:1029C00020E0E114F10441F084E1F801ABEDB2E064
:1029D00001900D928A95E1F76091030370E0660F14
:1029E000771F61517D4F45E08BED92E00E940D1500
:1029F000EF2819F40E94771302C081E090E06496FA
:102A00000FB6F894DEBF0FBECDBFDF91CF911F91FF
:102A10000F91FF90EF9008950895FF920F931F93E9
:102A2000CF93DF93F82E092F162FD72FC42F2223F1
:102A300049F081E0809380020E94722090937F028F
:102A400080937E02809180028823D9F080917E025B
:102A500090917F020E948A20059798F0EF2DF02F29
:102A6000A12FBD2F80E090E04C2F50E084179507F8
:102A700034F4219131912D933D930196F7CF10922B
:102A80008002DF91CF911F910F91FF9008952398BD
:102A90002B9883B183FB882780F908958091830266
:102AA00081110DC00E947A28811102C082E001C00C
:102AB00081E080938302823011F40E94752881E0C6
:102AC00090918302913009F080E008950E944715AB
:102AD000809304010E944E1581110C94C81508952D
:102AE0000E944E15811102C00C94CA15089581E010
:102AF000909184029A3008F080E00895EF92FF925E
:102B00000F931F93CF938C017B01C0918402CA3035
:102B100038F4B701C8010E941816811126C00AC0F6
:102B200080918102909182020E948A20843F91408C
:102B300080F719C0809184028F3F19F08F5F8093D6
:102B40008402809184028A30E0F00E947220909387
:102B500082028093810280917C0280FF04C088E71A
:102B600093E00E94090380E00DC0CA3040F08091DC
:102B70007C0280FF04C085E693E00E940903109266
:102B8000840281E0CF911F910F91FF90EF90089503
:102B90000C94821D0C94851DDF92EF92FF920F938F
:102BA0001F93CF93DF937901C82F880FDD0B411559
:102BB0005105A9F0FE0193E0EE0FFF1F9A95E1F792
:102BC000EB5FFE4F818192818B579D4F208130E0DA
:102BD0004217530708F49A01A9010E94CE28CE019A
:102BE0000E946E1ED82E8823D1F001151105B9F070
:102BF00083E0CC0FDD1F8A95E1F7FE01EB5FFE4F0E
:102C0000438150E00417150708F4A801CB5FDE4F9D
:102C10006C817D816B577D4FC7010E94CE288D2D21
:102C2000DF91CF911F910F91FF90EF90DF9008956A
:102C30000C9451170C9471170F931F93CF93DF933C
:102C400000D000D0CDB7DEB76091A6027091A70288
:102C50008091A8029091A9020E9499206436710582
:102C60008105910528F10E94AA12DC01CB01029690
:102C7000A11DB11D89839A83AB83BC8300E010E062
:102C800020E030E044E050E0BE016F5F7F4F82E023
:102C90000E94CC15182F882361F00E947E2060933B
:102CA000A6027093A7028093A8029093A90201C084
:102CB00011E0812F0F900F900F900F90DF91CF9127
:102CC0001F910F9108958F929F92AF92BF92CF92D2
:102CD000DF92EF92FF920F931F93CF93DF937C01CC
:102CE0005B01942E852E69010E947715811103C026
:102CF00001E010E002C00AE010E0C1E0D0E0F8948A
:102D0000B501C701F60109957894811129C0219672
:102D10000C171D078CF0CC9F9001CD9F300D300D0E
:102D2000112480E090E045E34A95F1F70000019618
:102D300028173907C1F7E3CF90917C02892F817062
:102D400090FF0FC08F929F928EEA93E09F938F9394
:102D50000E94A2030F900F900F900F9080E001C08F
:102D600081E0DF91CF911F910F91FF90EF90DF9065
:102D7000CF90BF90AF909F908F900895AF92BF92E9
:102D8000CF92DF92EF92FF920F931F93CF93DF9337
:102D9000CDB7DEB72B970FB6F894DEBF0FBECDBF11
:102DA0007B01C090A201D090A30101E010E09E0140
:102DB000255F3F4F40E050E060E070E080E00E941F
:102DC000CC15182F882309F43EC056018FEFA81A9E
:102DD000B80A6091A2027091A3028091A40290911E
:102DE000A5020E949920643671058105910518F1AC
:102DF0000AE010E09E012F5F3F4F40E050E060E0AE
:102E000070E081E00E94CC15182F6AE070E0C501E7
:102E10000E94D01A91E02B85281390E0192339F1F4
:102E20000E947E206093A2027093A3028093A4026A
:102E30009093A50211C06AE070E0C5010E94D01A0B
:102E40009B858913D5CF8AE0F6013196DE01119674
:102E500001900D928A95E1F7112349F08AE0FE0175
:102E60003196A8E9B2E001900D928A95E1F78AE0E7
:102E7000E8E9F2E0D70101900D928A95E1F7812F00
:102E80002B960FB6F894DEBF0FBECDBFDF91CF916A
:102E90001F910F91FF90EF90DF90CF90BF90AF9078
:102EA00008950F931F93CF93DF93EC018B012EEBCB
:102EB00036E144EA51E00E946316882361F02CE178
:102EC00036E141EB51E0B801CE01DF91CF911F9186
:102ED0000F910C94631680E0DF91CF911F910F91B9
:102EE00008950F931F93CF93DF93F894C091A2019D
:102EF000D091A301CE0101962AE0FB01DC010190F3
:102F00000D922A95E1F76AE070E00E94D01A88835A
:102F10007894F8946B857C858D859E8500919402CC
:102F200010919502209196023091970260177107D7
:102F30008207930751F060939402709395028093F7
:102F40009602909397020E948D127894DF91CF9110
:102F50001F910F9108950E943B230E94D00F0C9463
:102F600047230E944B230E947B100C9469230E94EC
:102F700010200E9422230E94BE0F0E94AB170E94C5
:102F8000B1170E94C80FFBCF8091B00280FF06C02E
:102F90006091220170E0660F771F26C081FF04C098
:102FA0006091220184E005C082FF07C06091220188
:102FB00088E0689FB001112417C09091AF02992357
:102FC000D1F060912101961788F72091220188E0C5
:102FD000289F90011124929FA001939F500D1124CE
:102FE00070E0CA010E9493286038710540F46115B1
:102FF000710519F406C068E070E0862F08958FE728
:10300000089581E008958091B00280FF08C060912A
:103010001E0170E0759567957595679521C081FFD4
:1030200006C060911E0170E07595679519C082FF1A
:1030300004C060911E0170E010C09091AE0299230F
:1030400099F060911D019617A0F780911E01899F4C
:10305000C001112470E00E9493286038710540F48B
:103060006115710519F406C061E070E0862F0895BE
:103070008FE7089581E008958D3E21F40E94C417E2
:10308000819504C08E3E29F40E94C4178093B40237
:1030900008958F3E21F40E94C417819504C0803F9B
:1030A00029F40E94C4178093B3020895893F19F44C
:1030B0000E94031805C08A3F31F40E9403188195CD
:1030C0008093B50208958B3F21F40E9403188195E7
:1030D00004C08C3F29F40E9403188093B60208951F
:1030E0009FE0980F983078F421E030E0A90102C009
:1030F000440F551F9A95E2F7CA019091B202892BAD
:103100008093B20208958D3F21F48091B0028160D6
:103110000BC08E3F21F48091B002826005C08F3FCA
:1031200029F48091B00284608093B00208958D3EAE
:1031300039F49091B40297FF35C01092B40259C08F
:103140008E3E29F49091B4021916BCF32BC09091D5
:10315000B3028F3E29F497FF25C01092B30249C0F5
:10316000803F19F41916CCF31DC09091B502893F28
:1031700029F41916BCF41092B5023BC08A3F19F429
:1031800097FF10C0F8CF8B3F39F49091B60297FFAC
:1031900009C01092B6022DC08C3F21F49091B60266
:1031A0001916BCF39FE0980F983080F421E030E0CE
:1031B000A90102C0440F551F9A95E2F7CA018095F4
:1031C0009091B20289238093B20213C08D3F21F403
:1031D0008091B0028E7F0BC08E3F21F48091B002AF
:1031E0008D7F05C08F3F29F48091B0028B7F809343
:1031F000B0028091B302811106C08091B4028111A6
:1032000002C01092AF028091B502811106C0809178
:10321000B602811102C01092AE02089580917C0224
:1032200083FF7EC08BEE93E00E9409038091B2027F
:103230001F928F9386EE93E09F938F930E94A20339
:1032400084EE93E00E9409038091B302282F082E98
:10325000000C330B3F938F9381EE93E09F938F93FA
:103260000E94A2038FED93E00E9409038091B402B3
:10327000282F082E000C330B3F938F938CED93E097
:103280009F938F930E94A2038AED93E00E9409030B
:103290008091B502282F082E000C330B3F938F939B
:1032A00087ED93E09F938F930E94A20385ED93E0B7
:1032B0000E9409038091B602282F082E000C330BC0
:1032C0003F938F9382ED93E09F938F930E94A2038D
:1032D0008FEC93E00E9409038091AF021F928F93BD
:1032E0008CEC93E09F938F930E94A2038AEC93E06F
:1032F0000E9409038091B0021F928F9387EC93E0A4
:103300009F938F930E94A20384EC93E00E94090391
:103310008DB79EB74C960FB6F8949EBF0FBE8DBF6B
:103320000E9472202091B302211104C02091B402A6
:10333000222321F09093AD028093AC022091B5023C
:10334000211104C02091B602222321F09093AB02F8
:103350008093AA0281EB92E00C944F1FEF92FF92B0
:103360000F931F93CF93DF9300D000D000D0CDB741
:10337000DEB786E0E1EBF2E0DE01119601900D92FE
:103380008A95E1F7E090B302F090B4020091B502A3
:103390001091B6021092B3021092B4021092B502CC
:1033A0001092B602E11003C0FF2009F45DC08091C5
:1033B000AC029091AD020E948A20AC019091AF02C4
:1033C000992339F02091230130E02417350758F074
:1033D0004BC0209124018AE0289F900111242417DA
:1033E000350718F041C09F3F19F09F5F9093AF02DF
:1033F000EE2061F00E94C4171E1414F09FEF01C06C
:1034000091E0989F902D11249093B302FF2061F0DA
:103410000E94C4171F1414F09FEF01C091E0989F01
:10342000902D11249093B4023091B3023323E1F034
:103430002091B4022223C1F045EB3403C0011124D2
:10344000992319F09093B30203C081E08093B302F3
:1034500035EB2303C0011124992319F09093B40292
:1034600003C081E08093B402011103C0112309F469
:103470005DC08091AA029091AB020E948A20AC01AB
:103480009091AE02992339F020911F0130E024176A
:10349000350758F04BC0209120018AE0289F900109
:1034A00011242417350718F041C09F3F19F09F5F82
:1034B0009093AE02002361F00E940318101614F0DE
:1034C0009FEF01C091E0989F902D11249093B50239
:1034D000112361F00E940318111614F09FEF01C030
:1034E00091E0989F902D11249093B6023091B502EF
:1034F0003323E1F02091B6022223C1F045EB3403DF
:10350000C0011124992319F09093B50203C081E002
:103510008093B50235EB2303C0011124992319F0E0
:103520009093B60203C081E08093B6028091B3020B
:1035300081110BC08091B402811107C08091B50246
:10354000811103C08091B60281110E940E19EB8295
:10355000FC820D831E8386E0FE013196A1EBB2E072
:1035600001900D928A95E1F726960FB6F894DEBF8A
:103570000FBECDBFDF91CF911F910F91FF90EF90C4
:103580000895E1EBF2E086E0DF011D928A95E9F70C
:103590001092AF021092AE021092B00208950895F8
:1035A000FC01680F791F8FEF91E3E617F70771F0C1
:1035B0002191822728E030E087FF03C0880F892708
:1035C00001C0880F21503109B9F7EFCF0895CF938B
:1035D000DF93EC01FB018281882309F43CC1C430F4
:1035E000FDE5DF0760F4CB3F9CE5D90788F49E0139
:1035F00022503C452431310508F02EC109C0C236A5
:10360000EDE5DE0729F0C63AFDE5DF0709F024C144
:103610000E94F90E9093D9028093D802C1318CE5B3
:10362000D80709F4C6C008F042C0C930ECE5DE078F
:1036300009F49BC000F5C5308CE5D80709F485C0B6
:1036400078F4C330ECE5DE0709F478C008F07AC0FE
:10365000C230DC4509F0F5C08091D8028160EFC02E
:10366000C7309CE5D90709F478C008F07AC080918A
:10367000D8028061E4C0CD30FCE5DF0709F487C0E3
:1036800058F4CB309CE5D90709F479C008F07BC029
:103690008091D80288606FC0CF30FCE5DF0709F465
:1036A00080C008F082C08091D802877FC8C0CE3F1A
:1036B0009CE5D90709F471C000F5C531FCE5DF07C9
:1036C00009F485C068F4C3319CE5D90709F475C0D5
:1036D00008F095C00E9496088091D8028F77AFC0FD
:1036E000CC3FFCE5DF07A9F108F054C0CB3FDC4537
:1036F00009F0A7C08091D90240C0C230EDE5DE07D5
:1037000009F489C058F4C1158DE5D80709F45AC0E9
:1037100008F069C08091D90282602FC0C236EDE501
:10372000DE0709F47CC0C63AFDE5DF0709F481C075
:10373000C330DD4509F085C080E06EC08091D802BD
:1037400082607DC08091D80216C08091D8028860C6
:1037500076C08091D90282604FC08091D802806289
:103760006EC08091D80280646AC00E9496088091E1
:10377000D802806864C0846062C081603DC080916E
:10378000D8028E7F5CC08091D8028D7F58C0809116
:10379000D80216C08091D90218C08091D9028D7FBD
:1037A0002BC08091D8028F7E4AC08091D8028F7D35
:1037B00046C08091D8028F7B42C08091D802877F1B
:1037C0008B7F3DC08091D9028D7F8E7F15C0809107
:1037D000D80282FB222720F991E0922790FB82F900
:1037E00090FB83F92CC08091D902982F909591700D
:1037F0008E7F892B90FB81F98093D90222C00E9491
:1038000096088091D80287FB222720F991E0922721
:1038100090FB87F914C081E00E94900F12C0809144
:10382000D80284FB222720F991E0922790FB84F9AB
:1038300006C08091D802982F909590FB80F98093D4
:10384000D8028091D8029091D9020E940A0F0E945A
:10385000960880E001C081E0DF91CF910895CF9379
:10386000DF9386319C4541F5EB010E94E90D982FCD
:103870008A812091020130910301882379F09A7A9C
:1038800081E009F480E08093B702911102C069E2FF
:1038900001C065E3C9010E94CB1F0AC08091B70235
:1038A000811102C069E201C065E3C9010E94CD1F18
:1038B0000E942B0E80E001C081E0DF91CF9108953E
:1038C0000F931F93CF93DF93C42FD22FFC018281DC
:1038D0008823C9F04093BA020E9472209093B902E3
:1038E0008093B80280E28C0F883008F057C0C77010
:1038F00081E001C0880FCA95EAF7DF91CF911F914F
:103900000F910C94F3058091BA02481330C0809156
:10391000B8029091B9020E948A20883C910538F53E
:1039200010E21D0FCD17B9F080E28C0F883040F403
:10393000C77081E001C0880FCA95EAF70E94FA05B6
:10394000183028F581E09D2F977001C0880F9A9557
:10395000EAF70E94F305802F0E94EA051830F0F480
:10396000D77081E001C0880FDA95EAF70AC080E2DB
:103970008C0F883098F4C77081E001C0880FCA9519
:10398000EAF7DF91CF911F910F910C94FA05802FE8
:10399000DF91CF911F910F910C94EA05DF91CF91A8
:1039A0001F910F9108950F939C01CB01243F4CE58B
:1039B000340731F188F4293DFCE53F07D9F02A3D71
:1039C0004CE5340779F1283D3C45A9F506E221EEA6
:1039D00041EE68ED7CE52BC0263FFCE53F07E1F0BA
:1039E000A8F0273F3C4539F507E225EE46EE67EFA4
:1039F0007CE51DC007E225EE45EE69ED7CE517C0CC
:103A000006E221EE40EE64EF7CE511C007E225EE10
:103A100044EE65EF7CE50BC006E221EE42EE66EF78
:103A20007CE505C008E221E045EE6AED7CE50E94F8
:103A3000601C80E008C0FC018281882319F010928C
:103A4000BA0201C081E00F9108958EE14A9B02C045
:103A50008150E1F74A9BFECF08955A9880E28A95FB
:103A6000F1F75A9A0895FC012AE02A95F1F728E027
:103A700090E080E031E040E14A95F1F7880F4A9B01
:103A800002C08160932700C0000040E14A95F1F731
:103A9000215089F720E12A95F1F729B100C00000F3
:103AA00030E13A95F1F722FB222720F99227208175
:103AB000920F90830895EF92FF920F931F93CF93ED
:103AC000DF931F92CDB7DEB719828C017C01E60E21
:103AD000F11C0E151F0551F00E94251DCE01019607
:103AE0000E94331DF80181938F01F3CF81E099810A
:103AF000911180E00F90DF91CF911F910F91FF9076
:103B0000EF900895529A5A9A089552985A9AEA9ABA
:103B1000E9E6F0E080818F7C80830895615091E038
:103B200001C0990F6A95EAF720E031E0992361F02E
:103B3000492F482319F05A9A232701C05A9840E286
:103B40004A95F1F79695F2CF222311F05A9A01C0C7
:103B50005A9880E28A95F1F75A980895FF920F9348
:103B60001F93CF93DF93EC018C01060F111DC0173B
:103B7000D10741F0F9900E942D1D68E08F2D0E9421
:103B80008E1DF5CFDF91CF911F910F91FF9008957A
:103B90001F920F920FB60F9211240F931F932F9322
:103BA0003F934F935F936F937F938F939F93AF93C5
:103BB000BF93EF93FF93CF93DF931F92CDB7DEB701
:103BC00019820E94251DCE0101960E94331D082FE7
:103BD000069506950695902F96959570202F257041
:103BE000920F292F237096959695920F87708913BF
:103BF0005FC0898181115CC0043008F059C080E148
:103C00008A95F1F75A9A529A82E08A95F1F700C0A4
:103C10005A9888E0089F80011124D801AB5FBE4FFD
:103C20001696ED91FC9117973097A9F06091A2013B
:103C30007091A30114962D913C911597260F371F73
:103C400011968D919C911297680F791F13964C9144
:103C500013978C910995F801EB5FFE4F6381662302
:103C600051F08091A2019091A30124813581820FAE
:103C7000931F0E94AE1D0E942D1D80E18A95F1F7D1
:103C80005A9852985A9A80E18A95F1F7F801EB5FB9
:103C9000FE4F6081662351F08091A2019091A301B3
:103CA00021813281820F931F0E945B1D0E94251D7E
:103CB0000F90DF91CF91FF91EF91BF91AF919F91C5
:103CC0008F917F916F915F914F913F912F911F91B4
:103CD0000F910F900FBE0F901F9018950F931F9389
:103CE000CF93DF93843091050CF06DC0EC01F89414
:103CF000529A5A9885E08A95F1F700009C2F969584
:103D000095702C2F2570920F892F8370969596951C
:103D100023E0CC0FDD1F2A95E1F7980F8E01092BC8
:103D20000E942D1D84E08A95F1F700C068E0802F85
:103D30000E948E1D80E18A95F1F752985A9A4A990D
:103D400002C000C0FCCF87E090E04A9B08C001970A
:103D500021F4529A5A9A789436C000C0F6CFFE01E8
:103D6000EB5FFE4F6381662381F08091A201909109
:103D7000A30124813581820F931F0E945B1D811155
:103D800004C0529A5A9A78941FC00E94251D80E25E
:103D90008A95F1F75A98529A80E18A95F1F7CB5FAC
:103DA000DE4F6881662351F08091A2019091A301BA
:103DB00029813A81820F931F0E94AE1D0E942D1D02
:103DC000789481E001C080E0DF91CF911F910F9145
:103DD00008959093CD018093CC0108959093C102F2
:103DE0008093C00208950E944E15811103C08091F6
:103DF000BB020895E091C002F091C102309721F01A
:103E00000190F081E02D099480E00895EF92FF92F7
:103E10000F931F93CF93DF93E091C002F091C10203
:103E20003097B1F18C010280F381E02D09958091EA
:103E30007C0282FF2DC080FF04C086E194E00E94D6
:103E40000903E80118E080E1E82E84E0F82E809173
:103E50007C0280FF0BC088811F928F93FF92EF92AC
:103E60000E94A2030F900F900F900F901150219677
:103E70001111EDCF80917C0280FF0AC08EE094E0AA
:103E8000DF91CF911F910F91FF90EF900C94090358
:103E9000DF91CF911F910F91FF90EF900895E091E6
:103EA000C002F091C102309739F022E0DC012C937E
:103EB0000480F581E02D099408952091BE0230918F
:103EC000BF022817390771F09093BF028093BE029A
:103ED000E091C002F091C102309721F00680F78195
:103EE000E02D099408952091BC023091BD0228175D
:103EF000390771F09093BD028093BC02E091C0023B
:103F0000F091C102309721F00084F185E02D0994F1
:103F10000895FC01329697E080E0915029F02191BC
:103F20002223D9F38F5FF9CF0895662349F0FC016E
:103F3000329608962191621729F0E817F907D1F710
:103F400080E0089581E008959C01FC0132969FEF86
:103F500080E04191461789F09F3F19F4411101C05B
:103F6000982F8F5F8630A9F79F3F39F0F901E90F4D
:103F7000F11D97FDFA956283089508959C012A5FCB
:103F80003F4FFC014281461301C012820196821705
:103F90009307B9F708950C94A41F0C94BE1F0296C2
:103FA00026E0FC0111922A95E9F7089508950C94F2
:103FB000D61F83E08093C2020C94D71F811102C0E8
:103FC00081E001C082E08093C2020C94D71F0C9460
:103FD000DE1F81E08093C2020C94D71F0C94E91F6E
:103FE00008950C94F01F0C94F11F0C94F01F0C9486
:103FF000F01F0C94F01FCF930E94F71F0E94B6147D
:104000000E94F51FC0E08C2F0E941413892B29F405
:10401000CF5FCA30C1F780E001C081E0CF91089541
:1040200008951F920F920FB60F9211248F939F93B2
:10403000AF93BF938091C302811113C08091040399
:1040400090910503A0910603B09107034196A11D2D
:10405000B11D8093040390930503A0930603B093CE
:104060000703BF91AF919F918F910F900FBE0F905B
:104070001F90189580910C03843031F10E948204C6
:104080001092C30220E488E190E00FB6F894A8955E
:10409000809360000FBE2093600083B7817F8460AF
:1040A00083BF83B7816083BF7894889583B78E7F01
:1040B00083BF0FB6F894A8958091600088618093C3
:1040C0006000109260000FBE08950E9496080C9444
:1040D000860482E084BD93E095BD9AEF97BD8093FE
:1040E0006E0008952FB7F894809104039091050312
:1040F000A0910603B09107032FBF08952FB7F8943E
:104100006091040370910503809106039091070369
:104110002FBF08959C014FB7F894809104039091AC
:104120000503A0910603B09107034FBF821B930BB9
:104130000895CF92DF92EF92FF922FB7F894C0903C
:104140000403D0900503E0900603F09007032FBF0F
:10415000A7019601261B370B480B590BCA01B90161
:10416000FF90EF90DF90CF90089578941F920F9278
:104170000FB60F9211248F939F93AF93BF938091AB
:10418000040390910503A0910603B09107030196E3
:10419000A11DB11D8093040390930503A093060312
:1041A000B0930703BF91AF919F918F910F900FBE76
:1041B0000F901F90189587E797E7909301088093D9
:1041C00000089AE088E10FB6F894A8958093600003
:1041D0000FBE90936000FFCF8091D20208950895A2
:1041E00022E02093E9002FEF3091E800215035FDC7
:1041F00006C035ED3A95F1F700002111F5CF209179
:10420000E80025FF0BC040E050E066E070E00E944F
:10421000D8238091E8008E778093E8000895CF93AB
:10422000DF9321E02093E9002FEF3091E800215047
:1042300035FD06C035ED3A95F1F700002111F5CFB7
:104240002091E80025FF14C0EC0140E050E068E058
:1042500070E00E94D8238091E8008E778093E80078
:1042600088E0FE01AAECB2E001900D928A95E1F798
:10427000DF91CF9108958093C6027093C802609336
:10428000C70280910C03843001F582E08093E9003D
:104290008FEF9091E800815095FD06C095ED9A95BD
:1042A000F1F700008111F5CF8091E80085FF0DC086
:1042B00040E050E063E070E086EC92E00E94D8239A
:1042C0008091E8008E778093E8000895BC0184E037
:1042D0000C943B21BC0183E00C943B218CE394E0E3
:1042E0000E94090380910B03811109C00E94692576
:1042F0000E94C6258091E20084608093E2000895C8
:1043000088E394E00E94090310920B03089584E36C
:1043100094E00E9409030C94EE1F80E394E00E9455
:1043200009036091080381E0611101C080E00C94F1
:10433000D91F8CE294E00E94090390910C0381E064
:10434000943009F080E0609108030C94DE1F209106
:10435000C5022F5F822F62E30E948728992319F0FC
:104360002093C50208951092C5028091C902882346
:1043700071F180910C03843041F58091E9008F70D8
:104380002091EC00922F917020FD90E8892B93E012
:104390009093E9009091EB0090FF14C09091EE0093
:1043A00097FF10C09091E80095FF03C01092F100B4
:1043B000F9CF9091E80090FF05C09091E8009E77BA
:1043C0009093E8008F708093E9001092C9020895DD
:1043D00042E061EC81E00E94E22442E261EC82E092
:1043E0000E94E22442E261EC83E00E94E224909188
:1043F0000C0381E0943009F080E0609108030C9494
:10440000E71F80910E03833009F461C030F48130DE
:1044100071F0823009F49AC008958A3009F486C098
:104420008B3009F46CC0893009F0A8C020C080919D
:104430000D03813A09F0A2C08091E800877F809344
:10444000E8008091110390911203892B21F468E018
:104450008AEC92E003C060E080E090E070E00E94AF
:1044600023248091E8008B778093E8000895809161
:104470000D03813209F082C08091110390911203E3
:10448000029708F07BC08091E800877F8093E80066
:104490008091E80082FD05C080910C038111F8CF66
:1044A0006DC02091F3008091F20090E0922B029772
:1044B00031F48091F100813011F0863021F4809147
:1044C000F1008093D2028091E8008B7753C08091F5
:1044D0000D03813A09F052C08091110390911203AB
:1044E000892B09F04BC08091E800877F8093E8001A
:1044F0008091E80080FFFCCF8091310136C080912F
:104500000D038132D9F58091110390911203892B0B
:10451000A9F58091E800877F8093E8000E94172525
:1045200080910F03809331010C94960880910D03C4
:10453000813221F58091E800877F8093E8000E9416
:104540001725809110038093D302089580910D0365
:10455000813AA1F48091E800877F8093E800809100
:10456000E80080FFFCCF8091D3028093F10080911E
:10457000E8008E778093E8000C94172508959FB784
:10458000F8941092C9029FBF90910C03943009F0E7
:1045900057C09091E9009F703091EC00232F21705B
:1045A00030FD20E8922B23E02093E9002091EB00DE
:1045B00020FF43C02091EE0027FF3FC02091C4029E
:1045C000222321F02091E80025FF37C01092C40279
:1045D00026E03091E80035FD15C030910C033430F1
:1045E00061F53091EB0035FD28C0215021F481E0C8
:1045F0008093C40222C0EFE9FFE03197F1F700C0D9
:104600000000E7CF8093F1008091E80085FD0AC0AB
:104610008091E80080FFFCCF8091E8008E77809346
:10462000E80006C08FB7F89421E02093C9028FBF3D
:104630009F709093E90080E008959F709093E90047
:104640008FEF089584B7877F84BF0FB6F894A8953D
:1046500080916000886180936000109260000FBEBE
:1046600090E080E80FB6F894809361009093610029
:104670000FBE0C94E91F0E9469250E94C625E2EE38
:10468000F0E080818460808378940C945A2885E2DD
:1046900091E00C94EE1E80910C038530C9F488E201
:1046A00094E00E94090380910C03853079F40E9404
:1046B0003A2080910A038823B1F30E94FB1F8823CC
:1046C00091F30E94C2230E949608EDCF0C946520BE
:1046D000089508950C946C23292F33272330310536
:1046E000C9F060F42130310581F02230310509F044
:1046F00041C08BE590E022E734E040C02132310533
:10470000E1F02232310531F135C082E190E02DEC4B
:1047100034E034C099278130910549F028F00297A0
:1047200049F5E0E4F4E005C0EEE6F4E002C0E0E5BF
:10473000F4E0849190E09F0121C063307105D0F4D2
:10474000660F771FFB01EB53FE4F2081318189E01B
:1047500090E014C06330710568F4FB01EE0FFF1F99
:10476000E154FE4F20813181FB01E454FE4F8081F2
:1047700090E004C080E090E020E030E0FA01318376
:104780002083089580E189BD82E189BD09B400FEDE
:10479000FDCF8091D8008F7D8093D8008091E0007C
:1047A00082608093E0008091E00081FDFCCF08955D
:1047B000CF92DF92EF92FF920F931F93CF93DF93ED
:1047C000EC018B017A010E943625811133C0E1147E
:1047D000F10439F0F70180819181081B190BC80F92
:1047E000D91FC12CD12C0115110519F18091E800B8
:1047F00085FD16C08091E8008E778093E800E11473
:10480000F10449F0F70180819181C80ED91ED1824F
:10481000C08285E00FC00E943625882321F30AC09C
:1048200089918093F10001501109FFEFCF1ADF0A3F
:10483000DACF80E0DF91CF911F910F91FF90EF9041
:10484000DF90CF9008952091130330911403261721
:10485000370748F06115710539F42091E8002E778B
:104860002093E80001C0B901FC0120E06115710549
:1048700079F180910C038823F1F18530F1F1809179
:10488000E80083FD3CC08091E80082FD2EC080914D
:10489000E80080FFEBCF2091F3008091F20090E0E0
:1048A000922B6115710551F08830910538F42191F2
:1048B0002093F100615071090196F3CF21E0089730
:1048C00009F020E08091E8008E778093E800CECF59
:1048D0002111CFCF0AC080910C03882361F085306D
:1048E00061F08091E80083FD0AC08091E80082FFBA
:1048F000F2CF80E0089582E0089583E0089581E09A
:10490000089520911303309114032617370748F0B8
:104910006115710539F42091E8002E772093E800A5
:1049200001C0B901FC0120E06115710591F1809190
:104930000C03882309F440C0853009F43FC08091FE
:10494000E80083FD3DC08091E80082FD2FC080918A
:10495000E80080FFE9CF2091F3008091F20090E021
:10496000922B6115710559F08830910540F424911E
:104970002093F1003196615071090196F2CF21E048
:10498000089709F020E08091E8008E778093E80096
:10499000CBCF2111CCCF0AC080910C03882361F0CA
:1049A000853061F08091E80083FD0AC08091E800C5
:1049B00082FFF2CF80E0089582E0089583E00895B9
:1049C00081E00895982F973068F59093E900981743
:1049D00039F07091EC002091ED005091F00003C08F
:1049E000242F762F50E021FD02C09F5FECCF309145
:1049F000EB003E7F3093EB003091ED003D7F309334
:104A0000ED003091EB0031603093EB007093EC00DF
:104A10002093ED005093F0002091EE0027FDE5CFAC
:104A200080E008958F708093E90081E0089580917F
:104A30000D0387FF11C08091E80082FD05C08091C1
:104A40000C038111F8CF11C08091E8008B770BC067
:104A500080910C03882349F08091E80080FFF8CF13
:104A60008091E8008E778093E80008952091E4001B
:104A70003091E50095E64091EC00842F817040FF75
:104A800023C08091E80080FD1DC080910C03882325
:104A900099F0853099F08091EB0085FD11C040912F
:104AA000E4005091E5002417350729F3915011F0E7
:104AB0009A01E1CF84E0089582E0089583E00895AB
:104AC00081E0089580E008954091E80042FFDDCF45
:104AD00008950E94D7250E94DF25E0EEF0E0808156
:104AE00081608083E8EDF0E080818F77808319BC5E
:104AF000A7EDB0E08C918E7F8C9380818F7E808338
:104B000010920B0308950F931F93CF93DF930E948E
:104B1000D7250E94DF25C8EDD0E088818F77888374
:104B200088818068888388818F7D888319BC1092F2
:104B30000C031092080310920A031092090300EE6E
:104B400010E0F80180818B7F808388818160888379
:104B500042E060E080E00E94E224E1EEF0E080814B
:104B60008E7F8083E2EEF0E08081816080838081AF
:104B700088608083F80180818E7F80838881806156
:104B80008883DF91CF911F910F910895E8EDF0E0B8
:104B900080818F7E8083E7EDF0E08081816080837B
:104BA00084E082BF81E080930B030C948325E8EDC1
:104BB000F0E080818E7F80831092E2000895109251
:104BC000DA001092E10008951F920F920FB60F9233
:104BD00011242F933F934F935F936F937F938F9302
:104BE0009F93AF93BF93EF93FF938091E10082FF78
:104BF0000BC08091E20082FF07C08091E1008B7FB3
:104C00008093E1000E94A7218091DA0080FF1FC0FD
:104C10008091D80080FF1BC08091DA008E7F809346
:104C2000DA008091D90080FF0DC080E189BD82E16A
:104C300089BD09B400FEFDCF81E080930C030E9482
:104C40006E2105C019BC10920C030E948021809136
:104C5000E10080FF19C08091E20080FF15C08091C3
:104C6000E2008E7F8093E2008091E2008061809379
:104C7000E2008091D80080628093D80019BC85E062
:104C800080930C030E948D218091E10084FF30C04D
:104C90008091E20084FF2CC080E189BD82E189BD62
:104CA00009B400FEFDCF8091D8008F7D8093D8009D
:104CB0008091E1008F7E8093E1008091E2008F7E01
:104CC0008093E2008091E20081608093E200809115
:104CD0000803882311F084E007C08091E30087FD7A
:104CE00002C081E001C083E080930C030E949921FF
:104CF0008091E10083FF29C08091E20083FF25C0FD
:104D00008091E100877F8093E10082E080930C0333
:104D1000109208038091E1008E7F8093E1008091E2
:104D2000E2008E7F8093E2008091E20080618093B8
:104D3000E20042E060E080E00E94E2248091F00026
:104D400088608093F0000E948721FF91EF91BF91CE
:104D5000AF919F918F917F916F915F914F913F9113
:104D60002F910F900FBE0F901F9018951F920F92CA
:104D70000FB60F9211242F933F934F935F936F932E
:104D80007F938F939F93AF93BF93CF93DF93EF93D3
:104D9000FF93C091E900CF708091EC00D82FD170C3
:104DA00080FDD0E81092E9008091F000877F809329
:104DB000F00078940E94FA261092E9008091F000A9
:104DC00088608093F000CD2BCF70C093E900FF91F5
:104DD000EF91DF91CF91BF91AF919F918F917F9193
:104DE0006F915F914F913F912F910F900FBE0F9058
:104DF0001F9018951F93CF93DF93CDB7DEB7AA9777
:104E00000FB6F894DEBF0FBECDBFEDE0F3E08091AA
:104E1000F100819323E0E531F207C9F70E940122F6
:104E20008091E80083FF2EC180910D0390910E03C5
:104E3000492F50E04A30510508F024C1FA01EE59DB
:104E4000FF4F0C94A728803821F0823809F01AC14E
:104E500008C08091090390910A03992389F0826028
:104E60000FC0809111038F70873008F00BC18093C1
:104E7000E9008091EB0085FB882780F91092E9001A
:104E80009091E800977F9093E8008093F100109252
:104E9000F100D1C0282F2D7F09F0F4C0882319F02C
:104EA000823061F0EFC080910F03813009F0EAC0D9
:104EB000933009F080E080930A032EC080910F03A5
:104EC00081112AC0809111038F702FEF280F263097
:104ED00008F0D8C08093E9002091EB0020FF1CC0AF
:104EE000933021F48091EB00806214C09091EB002C
:104EF00090619093EB0021E030E0A90102C0440FE3
:104F0000551F8A95E2F74093EA001092EA008091DB
:104F1000EB0088608093EB001092E9008091E8003C
:104F2000877F8093E8000E941725ACC08111AAC03A
:104F300010910F031F778091E3008078812B80937D
:104F4000E3008091E800877F8093E8000E941725A6
:104F50008091E80080FFFCCF8091E300806880931F
:104F6000E300111102C082E001C083E080930C03D2
:104F700089C08058823008F085C080910F039091DD
:104F800010038C3D53E0950779F583E08A838AE22C
:104F900089834FB7F894DE01139620E03EE051E29A
:104FA000E32FF0E050935700E49120FF03C0E29517
:104FB000EF703F5FEF708E2F90E0EA3010F0C796F1
:104FC00001C0C0968D939D932F5F243149F74FBF49
:104FD0008091E800877F8093E8006AE270E0CE016C
:104FE00001960E94232416C0609111037091120350
:104FF000AE014F5F5F4F0E946A23BC01892B09F409
:1050000041C09091E800977F9093E80089819A8150
:105010000E9481248091E8008B778093E80032C061
:10502000803881F58091E800877F8093E800809147
:1050300008038093F1008091E8008E7772CF811190
:1050400021C080910F039091100399270297D4F407
:105050008091E800877F8093E80080910F03809320
:1050600008030E94172580910803811106C08091D2
:10507000E30087FD02C081E001C084E080930C035F
:105080000E94E8218091E80083FF0AC08091E80037
:10509000877F8093E8008091EB0080628093EB0033
:1050A000AA960FB6F894DEBF0FBECDBFDF91CF91A9
:1050B0001F910895CF9380910C038823A1F0C09194
:1050C000E900CF709091EC00892F817090FD80E80D
:1050D000C82B1092E9008091E80083FD0E94FA2617
:1050E000CF70C093E900CF9108950E946925109276
:1050F0000C030895E8EDF0E08081806180838AE10F
:105100008A95F1F700C08091D90081700895991BAC
:1051100079E004C0991F961708F0961B881F7A95AE
:10512000C9F78095089597FB072E16F4009407D0D1
:1051300077FD09D00E94AD2807FC05D03EF490957C
:1051400081959F4F0895709561957F4F0895EE0F5B
:10515000FF1F0590F491E02D0994AA1BBB1B51E1A0
:1051600007C0AA1FBB1FA617B70710F0A61BB70BD7
:10517000881F991F5A95A9F780959095BC01CD017C
:105180000895FB01DC0104C08D910190801921F488
:1051900041505040C8F7881B990B0895FB01DC0172
:1051A00002C001900D9241505040D8F70895F999EE
:1051B000FECF92BD81BDF89A992780B50895A8E1E8
:1051C000B0E042E050E00C940B29262FF999FECF75
:1051D00092BD81BDF89A019700B4021639F01FBA4A
:1051E00020BD0FB6F894FA9AF99A0FBE0895039667
:1051F000272F0E94E6280E94E528252F0E94E628F6
:10520000242F0C94E6280196272F0E94E6280C9460
:10521000E528DC01CB01FC01F999FECF06C0F2BD07
:10522000E1BDF89A319600B40D9241505040B8F764
:065230000895F894FFCF81
:10523600C800560201000000010000000000000046
:105246000A01000000040B000000000000280850BE
:10525600011E0A1401EC200F21F0206A216621EFBD
:105266002001E200E900EA00B500B600B700CD0073
:105276008301CC008A0192019401210223022402B7
:105286002502260227022A02B300B4006F0070002E
:10529600818283E200E900EA00B500B600B700CDDE
:1052A600008301CC008A0192019401210223022489
:1052B600022502260227022A02B300B4006F0070FC
:1052C60000818283329190946697C63435F4F5F660
:1052D600F7318502736C6176655F6D61747269780A
:1052E6000073796E635F74696D657200407B227C22
:0C52F600050105DF0484049D04B60400DB
:00000001FF
